:047C00000C942A3E78
:147C540001E005BF02E005BFCFE5D8E0CDBFDEBFC051D0401B
:147C68000AEA08830024E0E6F0E010E0E23EF10711F0019233
:147C7C00FBCF0083E4E5FCE7A0E6B0E01CE7E435F10721F0C0
:147C9000C89531960D92F9CFF8D0FFCF05E4E8D00EE6E6D074
:147CA40003E6E4D003E5E2D0DFD001E2DFD019C01AD0809180
:147CB8006000909161008038EFEF9E0709F437D03DD0002367
:147CCC0051F062D094D0002319F001E2CBD005C000E4C8D0E2
:147CE00002C000E4C5D0E6CF0895BAD00023E9F3BDD0202E9F
:147CF4003324322C22243092610020926000AED00023E9F3CF
:147D0800B1D0202E33244090600050906100420C531C509231
:147D1C0061004092600027E030E082010E94B33F109361008E
:147D300000936000089581E08BBF22242BBE0C940000089598
:147D44000E94983F66274427AA2412C087D00023E9F38AD06A
:147D580082E690E0EA2DFF27E80FF91F0083EA2DFF27E80F3C
:147D6C00F91F2080620DA3948A2D803858F372D00023E9F3AA
:147D800075D0402F601711F401E001C000270E94913F0895E7
:147D94000E949A3F66271AC083E690E0E62FFF27E80FF91FD6
:147DA80020803324322C222482E690E0E62FFF27E80FF91F0A
:147DBC0040815527420D531D262F33278A010E94683F6E5F67
:147DD000603820F323E000916000109161000E94613F25E0B7
:147DE40000916000109161000E94613F0E94833F0E948E3F83
:147DF80008950E94983FAA2428C022272A2C332400916000C4
:147E0C0010916100020D131D0E94723FB80183E690E0EA2D25
:147E2000FF27E80FF91F20803324322C222482E690E0EA2D8F
:147E3400FF27E80FF91F40815527420D531D0417150711F0D1
:147E4800002707C08A2D8E5FA82E8A2D8038A8F201E00E9432
:147E5C00913F08955F9B02C001E001C0002708950CB1089529
:147E70005D9BFECF0CB90895002711270F5F1F4F0030EDE798
:147E84001E07D4F30895F89481E082BB22242AB82BB886E8BE
:147E980080BD20BC88E18AB944270BC049B9E2DF0EE3E2DF66
:147EAC00E5DFDEDF0C3311F4F3DE3FDF43954F3F98F33BDF03
:147EC000089527D0F12FE02F20935700E895089520D0F32FB5
:147ED400E22F112E002E31E030935700E8950895F12FE02FA8
:147EE80020FD20935700C895002DE395C895102D0895002EF8
:147EFC0019E010935700E895089505D0B1E1B0935700E895E7
:147F10000895B0915700B0FDFCCF0895E2E00C94A03FE4E00E
:147F24000C94A03FFA92EA92DA92CA92BA92AA927A936A9368
:147F38005A934A930895E1E049915991E0FD089569917991CB
:147F4C00E1FD0895A990B990E2FD0895C990D990E3FD089569
:147F6000E990F9900895222321F0000F111F2A95FACF0895B4
:00000001FF
